:0200000480007A
:100000006F00C004732F2034930F8000630AFF0336
:10001000930F90006306FF03930FB0006302FF038A
:10002000170F0080130F0FFE63040F0067000F000F
:10003000732F203463540F006F004000136E9E53E3
:10004000171F00002320CFFD6FF09FFF732540F1A5
:100050006310050073251030635805000F00F00F82
:10006000130E100073000000130E00009702000032
:10007000938282F973905230735020307350303035
:1000800073504030970200809382C2F7638C020065
:10009000739052109302B01A739022307323203061
:1000A000E39E62F873500030970200009382420191
:1000B00073901234732540F17300203093000000D8
:1000C00013010000B3812000930E0000130E2000E6
:1000D0006396D14D9300100013011000B3812000EE
:1000E000930E2000130E3000639AD14B9300300022
:1000F00013017000B3812000930EA000130E400086
:10010000639ED149930000003781FFFFB381200037
:10011000B78EFFFF130E50006392D149B7000080E5
:1001200013010000B3812000B70E0080130E6000A1
:100130006396D147B70000803781FFFFB38120006D
:10014000B78EFF7F130E7000639AD14593000000B5
:10015000378100001301F1FFB3812000B78E00004A
:10016000938EFEFF130E8000639AD143B700008088
:100170009380F0FF13010000B3812000B70E0080D0
:10018000938EFEFF130E9000639AD141B70000805A
:100190009380F0FF378100001301F1FFB38120004D
:1001A000B78E0080938EEEFF130EA0006398D13FB0
:1001B000B7000080378100001301F1FFB3812000F8
:1001C000B78E0080938EFEFF130EB0006398D13D72
:1001D000B70000809380F0FF3781FFFFB3812000DC
:1001E000B78EFF7F938EFEFF130EC0006398D13B46
:1001F000930000001301F0FFB3812000930EF0FF85
:10020000130ED000639CD1399300F0FF130110004E
:10021000B3812000930E0000130EE0006390D139EB
:100220009300F0FF1301F0FFB3812000930EE0FF75
:10023000130EF0006394D137930010003701008053
:100240001301F1FFB3812000B70E0080130E0001EF
:100250006396D1359300D0001301B000B380200025
:10026000930E8001130E1001639AD0339300E000C7
:100270001301B00033812000930E9001130E200172
:10028000631ED1319300D000B3801000930EA00103
:10029000130E30016394D031130200009300D0009C
:1002A0001301B000B3812000138301001302120078
:1002B00093022000E31452FE930E8001130E4001BE
:1002C000631ED32D130200009300E0001301B00061
:1002D000B3812000130000001383010013021200F9
:1002E00093022000E31252FE930E9001130E500170
:1002F0006316D32B130200009300F0001301B0002B
:10030000B3812000130000001300000013830100DC
:100310001302120093022000E31052FE930EA0017C
:10032000130E6001631CD327130200009300D0005A
:100330001301B000B38120001302120093022000C9
:10034000E31652FE930E8001130E70016398D125BF
:10035000130200009300E0001301B000130000003E
:10036000B38120001302120093022000E31452FE16
:10037000930E9001130E80016392D12313020000AB
:100380009300F0001301B000130000001300000000
:10039000B38120001302120093022000E31252FEE8
:1003A000930EA001130E9001639AD11F1302000057
:1003B0009300D000130000001301B000B3812000AF
:1003C0001302120093022000E31452FE930E8001E8
:1003D000130EA0016394D11D130200009300E000EE
:1003E000130000001301B00013000000B3812000CF
:1003F0001302120093022000E31252FE930E9001AA
:10040000130EB001639CD119130200009300F00099
:1004100013000000130000001301B000B38120009E
:100420001302120093022000E31252FE930EA00169
:10043000130EC0016394D117130200001301B00022
:100440009300D000B3812000130212009302200019
:10045000E31652FE930E8001130ED0016390D11566
:10046000130200001301B0009300E000130000002D
:10047000B38120001302120093022000E31452FE05
:10048000930E9001130EE001639AD1111302000044
:100490001301B0009300F0001300000013000000EF
:1004A000B38120001302120093022000E31252FED7
:1004B000930EA001130EF0016392D10F13020000FE
:1004C0001301B000130000009300D000B38120009E
:1004D0001302120093022000E31452FE930E8001D7
:1004E000130E0002639CD10B130200001301B00035
:1004F000130000009300E00013000000B38120000F
:100500001302120093022000E31252FE930E900198
:10051000130E10026394D109130200001301B000FE
:1005200013000000130000009300F000B3812000CE
:100530001302120093022000E31252FE930EA00158
:10054000130E2002639CD1059300F00033011000CC
:10055000930EF000130E30026312D10593000002D7
:1005600033810000930E0002130E40026318D10382
:10057000B3000000930E0000130E50026390D003EE
:10058000930000011301E00133802000930E00006E
:10059000130E60026314D001631CC0010F00F00F42
:1005A00063000E00131E1E00136E1E007300000079
:1005B0000F00F00F130E100073000000731000C046
:0405C0000000000037
:1010000000000000000000000000000000000000E0
:1010100000000000000000000000000000000000D0
:1010200000000000000000000000000000000000C0
:1010300000000000000000000000000000000000B0
:081040000000000000000000A8
:040000058000200057
:00000001FF
